
D:\STM32\Program\1.11_Odchudzanie\um0427\FWLib\project\RIDE\STM3210E-EVAL\stm32f10x_i2c.o:     file format elf32-littlearm
D:\STM32\Program\1.11_Odchudzanie\um0427\FWLib\project\RIDE\STM3210E-EVAL\stm32f10x_i2c.o

Disassembly of section .text.I2C_StructInit:

00000000 <I2C_StructInit>:
I2C_StructInit():
D:\STM32\Program\1.11_Odchudzanie\um0427\FWLib\library\src/stm32f10x_i2c.c:264
   0:	2300      	movs	r3, #0
   2:	8003      	strh	r3, [r0, #0]
D:\STM32\Program\1.11_Odchudzanie\um0427\FWLib\library\src/stm32f10x_i2c.c:270
   4:	8083      	strh	r3, [r0, #4]
D:\STM32\Program\1.11_Odchudzanie\um0427\FWLib\library\src/stm32f10x_i2c.c:273
   6:	80c3      	strh	r3, [r0, #6]
D:\STM32\Program\1.11_Odchudzanie\um0427\FWLib\library\src/stm32f10x_i2c.c:276
   8:	f44f 4380 	mov.w	r3, #16384	; 0x4000
D:\STM32\Program\1.11_Odchudzanie\um0427\FWLib\library\src/stm32f10x_i2c.c:267
   c:	f64b 72ff 	movw	r2, #49151	; 0xbfff
D:\STM32\Program\1.11_Odchudzanie\um0427\FWLib\library\src/stm32f10x_i2c.c:276
  10:	8103      	strh	r3, [r0, #8]
D:\STM32\Program\1.11_Odchudzanie\um0427\FWLib\library\src/stm32f10x_i2c.c:279
  12:	f241 3388 	movw	r3, #5000	; 0x1388
D:\STM32\Program\1.11_Odchudzanie\um0427\FWLib\library\src/stm32f10x_i2c.c:267
  16:	8042      	strh	r2, [r0, #2]
D:\STM32\Program\1.11_Odchudzanie\um0427\FWLib\library\src/stm32f10x_i2c.c:279
  18:	60c3      	str	r3, [r0, #12]
D:\STM32\Program\1.11_Odchudzanie\um0427\FWLib\library\src/stm32f10x_i2c.c:280
  1a:	4770      	bx	lr
Disassembly of section .text.I2C_Cmd:

00000000 <I2C_Cmd>:
I2C_Cmd():
D:\STM32\Program\1.11_Odchudzanie\um0427\FWLib\library\src/stm32f10x_i2c.c:297
   0:	b121      	cbz	r1, c <I2C_Cmd+0xc>
D:\STM32\Program\1.11_Odchudzanie\um0427\FWLib\library\src/stm32f10x_i2c.c:300
   2:	8803      	ldrh	r3, [r0, #0]
   4:	b29b      	uxth	r3, r3
   6:	f043 0301 	orr.w	r3, r3, #1	; 0x1
   a:	e004      	b.n	16 <I2C_Cmd+0x16>
D:\STM32\Program\1.11_Odchudzanie\um0427\FWLib\library\src/stm32f10x_i2c.c:305
   c:	8803      	ldrh	r3, [r0, #0]
   e:	f023 0301 	bic.w	r3, r3, #1	; 0x1
  12:	041b      	lsls	r3, r3, #16
  14:	0c1b      	lsrs	r3, r3, #16
  16:	8003      	strh	r3, [r0, #0]
D:\STM32\Program\1.11_Odchudzanie\um0427\FWLib\library\src/stm32f10x_i2c.c:307
  18:	4770      	bx	lr
  1a:	46c0      	nop			(mov r8, r8)
Disassembly of section .text.I2C_DMACmd:

00000000 <I2C_DMACmd>:
I2C_DMACmd():
D:\STM32\Program\1.11_Odchudzanie\um0427\FWLib\library\src/stm32f10x_i2c.c:324
   0:	b121      	cbz	r1, c <I2C_DMACmd+0xc>
D:\STM32\Program\1.11_Odchudzanie\um0427\FWLib\library\src/stm32f10x_i2c.c:327
   2:	8883      	ldrh	r3, [r0, #4]
   4:	b29b      	uxth	r3, r3
   6:	f443 6300 	orr.w	r3, r3, #2048	; 0x800
   a:	e004      	b.n	16 <I2C_DMACmd+0x16>
D:\STM32\Program\1.11_Odchudzanie\um0427\FWLib\library\src/stm32f10x_i2c.c:332
   c:	8883      	ldrh	r3, [r0, #4]
   e:	f423 6300 	bic.w	r3, r3, #2048	; 0x800
  12:	041b      	lsls	r3, r3, #16
  14:	0c1b      	lsrs	r3, r3, #16
  16:	8083      	strh	r3, [r0, #4]
D:\STM32\Program\1.11_Odchudzanie\um0427\FWLib\library\src/stm32f10x_i2c.c:334
  18:	4770      	bx	lr
  1a:	46c0      	nop			(mov r8, r8)
Disassembly of section .text.I2C_DMALastTransferCmd:

00000000 <I2C_DMALastTransferCmd>:
I2C_DMALastTransferCmd():
D:\STM32\Program\1.11_Odchudzanie\um0427\FWLib\library\src/stm32f10x_i2c.c:351
   0:	b121      	cbz	r1, c <I2C_DMALastTransferCmd+0xc>
D:\STM32\Program\1.11_Odchudzanie\um0427\FWLib\library\src/stm32f10x_i2c.c:354
   2:	8883      	ldrh	r3, [r0, #4]
   4:	b29b      	uxth	r3, r3
   6:	f443 5380 	orr.w	r3, r3, #4096	; 0x1000
   a:	e004      	b.n	16 <I2C_DMALastTransferCmd+0x16>
D:\STM32\Program\1.11_Odchudzanie\um0427\FWLib\library\src/stm32f10x_i2c.c:359
   c:	8883      	ldrh	r3, [r0, #4]
   e:	f423 5380 	bic.w	r3, r3, #4096	; 0x1000
  12:	041b      	lsls	r3, r3, #16
  14:	0c1b      	lsrs	r3, r3, #16
  16:	8083      	strh	r3, [r0, #4]
D:\STM32\Program\1.11_Odchudzanie\um0427\FWLib\library\src/stm32f10x_i2c.c:361
  18:	4770      	bx	lr
  1a:	46c0      	nop			(mov r8, r8)
Disassembly of section .text.I2C_GenerateSTART:

00000000 <I2C_GenerateSTART>:
I2C_GenerateSTART():
D:\STM32\Program\1.11_Odchudzanie\um0427\FWLib\library\src/stm32f10x_i2c.c:378
   0:	b121      	cbz	r1, c <I2C_GenerateSTART+0xc>
D:\STM32\Program\1.11_Odchudzanie\um0427\FWLib\library\src/stm32f10x_i2c.c:381
   2:	8803      	ldrh	r3, [r0, #0]
   4:	b29b      	uxth	r3, r3
   6:	f443 7380 	orr.w	r3, r3, #256	; 0x100
   a:	e004      	b.n	16 <I2C_GenerateSTART+0x16>
D:\STM32\Program\1.11_Odchudzanie\um0427\FWLib\library\src/stm32f10x_i2c.c:386
   c:	8803      	ldrh	r3, [r0, #0]
   e:	f423 7380 	bic.w	r3, r3, #256	; 0x100
  12:	041b      	lsls	r3, r3, #16
  14:	0c1b      	lsrs	r3, r3, #16
  16:	8003      	strh	r3, [r0, #0]
D:\STM32\Program\1.11_Odchudzanie\um0427\FWLib\library\src/stm32f10x_i2c.c:388
  18:	4770      	bx	lr
  1a:	46c0      	nop			(mov r8, r8)
Disassembly of section .text.I2C_GenerateSTOP:

00000000 <I2C_GenerateSTOP>:
I2C_GenerateSTOP():
D:\STM32\Program\1.11_Odchudzanie\um0427\FWLib\library\src/stm32f10x_i2c.c:405
   0:	b121      	cbz	r1, c <I2C_GenerateSTOP+0xc>
D:\STM32\Program\1.11_Odchudzanie\um0427\FWLib\library\src/stm32f10x_i2c.c:408
   2:	8803      	ldrh	r3, [r0, #0]
   4:	b29b      	uxth	r3, r3
   6:	f443 7300 	orr.w	r3, r3, #512	; 0x200
   a:	e004      	b.n	16 <I2C_GenerateSTOP+0x16>
D:\STM32\Program\1.11_Odchudzanie\um0427\FWLib\library\src/stm32f10x_i2c.c:413
   c:	8803      	ldrh	r3, [r0, #0]
   e:	f423 7300 	bic.w	r3, r3, #512	; 0x200
  12:	041b      	lsls	r3, r3, #16
  14:	0c1b      	lsrs	r3, r3, #16
  16:	8003      	strh	r3, [r0, #0]
D:\STM32\Program\1.11_Odchudzanie\um0427\FWLib\library\src/stm32f10x_i2c.c:415
  18:	4770      	bx	lr
  1a:	46c0      	nop			(mov r8, r8)
Disassembly of section .text.I2C_AcknowledgeConfig:

00000000 <I2C_AcknowledgeConfig>:
I2C_AcknowledgeConfig():
D:\STM32\Program\1.11_Odchudzanie\um0427\FWLib\library\src/stm32f10x_i2c.c:432
   0:	b121      	cbz	r1, c <I2C_AcknowledgeConfig+0xc>
D:\STM32\Program\1.11_Odchudzanie\um0427\FWLib\library\src/stm32f10x_i2c.c:435
   2:	8803      	ldrh	r3, [r0, #0]
   4:	b29b      	uxth	r3, r3
   6:	f443 6380 	orr.w	r3, r3, #1024	; 0x400
   a:	e004      	b.n	16 <I2C_AcknowledgeConfig+0x16>
D:\STM32\Program\1.11_Odchudzanie\um0427\FWLib\library\src/stm32f10x_i2c.c:440
   c:	8803      	ldrh	r3, [r0, #0]
   e:	f423 6380 	bic.w	r3, r3, #1024	; 0x400
  12:	041b      	lsls	r3, r3, #16
  14:	0c1b      	lsrs	r3, r3, #16
  16:	8003      	strh	r3, [r0, #0]
D:\STM32\Program\1.11_Odchudzanie\um0427\FWLib\library\src/stm32f10x_i2c.c:442
  18:	4770      	bx	lr
  1a:	46c0      	nop			(mov r8, r8)
Disassembly of section .text.I2C_OwnAddress2Config:

00000000 <I2C_OwnAddress2Config>:
I2C_OwnAddress2Config():
D:\STM32\Program\1.11_Odchudzanie\um0427\FWLib\library\src/stm32f10x_i2c.c:460
   0:	8983      	ldrh	r3, [r0, #12]
D:\STM32\Program\1.11_Odchudzanie\um0427\FWLib\library\src/stm32f10x_i2c.c:464
   2:	f001 01fe 	and.w	r1, r1, #254	; 0xfe
   6:	f023 03fe 	bic.w	r3, r3, #254	; 0xfe
   a:	041b      	lsls	r3, r3, #16
   c:	0c1b      	lsrs	r3, r3, #16
   e:	4319      	orrs	r1, r3
D:\STM32\Program\1.11_Odchudzanie\um0427\FWLib\library\src/stm32f10x_i2c.c:466
  10:	8181      	strh	r1, [r0, #12]
D:\STM32\Program\1.11_Odchudzanie\um0427\FWLib\library\src/stm32f10x_i2c.c:467
  12:	4770      	bx	lr
Disassembly of section .text.I2C_DualAddressCmd:

00000000 <I2C_DualAddressCmd>:
I2C_DualAddressCmd():
D:\STM32\Program\1.11_Odchudzanie\um0427\FWLib\library\src/stm32f10x_i2c.c:484
   0:	b121      	cbz	r1, c <I2C_DualAddressCmd+0xc>
D:\STM32\Program\1.11_Odchudzanie\um0427\FWLib\library\src/stm32f10x_i2c.c:487
   2:	8983      	ldrh	r3, [r0, #12]
   4:	b29b      	uxth	r3, r3
   6:	f043 0301 	orr.w	r3, r3, #1	; 0x1
   a:	e004      	b.n	16 <I2C_DualAddressCmd+0x16>
D:\STM32\Program\1.11_Odchudzanie\um0427\FWLib\library\src/stm32f10x_i2c.c:492
   c:	8983      	ldrh	r3, [r0, #12]
   e:	f023 0301 	bic.w	r3, r3, #1	; 0x1
  12:	041b      	lsls	r3, r3, #16
  14:	0c1b      	lsrs	r3, r3, #16
  16:	8183      	strh	r3, [r0, #12]
D:\STM32\Program\1.11_Odchudzanie\um0427\FWLib\library\src/stm32f10x_i2c.c:494
  18:	4770      	bx	lr
  1a:	46c0      	nop			(mov r8, r8)
Disassembly of section .text.I2C_GeneralCallCmd:

00000000 <I2C_GeneralCallCmd>:
I2C_GeneralCallCmd():
D:\STM32\Program\1.11_Odchudzanie\um0427\FWLib\library\src/stm32f10x_i2c.c:511
   0:	b121      	cbz	r1, c <I2C_GeneralCallCmd+0xc>
D:\STM32\Program\1.11_Odchudzanie\um0427\FWLib\library\src/stm32f10x_i2c.c:514
   2:	8803      	ldrh	r3, [r0, #0]
   4:	b29b      	uxth	r3, r3
   6:	f043 0340 	orr.w	r3, r3, #64	; 0x40
   a:	e004      	b.n	16 <I2C_GeneralCallCmd+0x16>
D:\STM32\Program\1.11_Odchudzanie\um0427\FWLib\library\src/stm32f10x_i2c.c:519
   c:	8803      	ldrh	r3, [r0, #0]
   e:	f023 0340 	bic.w	r3, r3, #64	; 0x40
  12:	041b      	lsls	r3, r3, #16
  14:	0c1b      	lsrs	r3, r3, #16
  16:	8003      	strh	r3, [r0, #0]
D:\STM32\Program\1.11_Odchudzanie\um0427\FWLib\library\src/stm32f10x_i2c.c:521
  18:	4770      	bx	lr
  1a:	46c0      	nop			(mov r8, r8)
Disassembly of section .text.I2C_ITConfig:

00000000 <I2C_ITConfig>:
I2C_ITConfig():
D:\STM32\Program\1.11_Odchudzanie\um0427\FWLib\library\src/stm32f10x_i2c.c:545
   0:	b122      	cbz	r2, c <I2C_ITConfig+0xc>
D:\STM32\Program\1.11_Odchudzanie\um0427\FWLib\library\src/stm32f10x_i2c.c:548
   2:	8883      	ldrh	r3, [r0, #4]
   4:	b29b      	uxth	r3, r3
   6:	ea41 0303 	orr.w	r3, r1, r3
   a:	e003      	b.n	14 <I2C_ITConfig+0x14>
D:\STM32\Program\1.11_Odchudzanie\um0427\FWLib\library\src/stm32f10x_i2c.c:553
   c:	8883      	ldrh	r3, [r0, #4]
   e:	b29b      	uxth	r3, r3
  10:	ea23 0301 	bic.w	r3, r3, r1
  14:	8083      	strh	r3, [r0, #4]
D:\STM32\Program\1.11_Odchudzanie\um0427\FWLib\library\src/stm32f10x_i2c.c:555
  16:	4770      	bx	lr
Disassembly of section .text.I2C_SendData:

00000000 <I2C_SendData>:
I2C_SendData():
D:\STM32\Program\1.11_Odchudzanie\um0427\FWLib\library\src/stm32f10x_i2c.c:571
   0:	8201      	strh	r1, [r0, #16]
D:\STM32\Program\1.11_Odchudzanie\um0427\FWLib\library\src/stm32f10x_i2c.c:572
   2:	4770      	bx	lr
Disassembly of section .text.I2C_ReceiveData:

00000000 <I2C_ReceiveData>:
I2C_ReceiveData():
D:\STM32\Program\1.11_Odchudzanie\um0427\FWLib\library\src/stm32f10x_i2c.c:587
   0:	8a00      	ldrh	r0, [r0, #16]
D:\STM32\Program\1.11_Odchudzanie\um0427\FWLib\library\src/stm32f10x_i2c.c:588
   2:	b2c0      	uxtb	r0, r0
   4:	4770      	bx	lr
   6:	46c0      	nop			(mov r8, r8)
Disassembly of section .text.I2C_Send7bitAddress:

00000000 <I2C_Send7bitAddress>:
I2C_Send7bitAddress():
D:\STM32\Program\1.11_Odchudzanie\um0427\FWLib\library\src/stm32f10x_i2c.c:610
   0:	b112      	cbz	r2, 8 <I2C_Send7bitAddress+0x8>
D:\STM32\Program\1.11_Odchudzanie\um0427\FWLib\library\src/stm32f10x_i2c.c:613
   2:	f041 0101 	orr.w	r1, r1, #1	; 0x1
   6:	e001      	b.n	c <I2C_Send7bitAddress+0xc>
D:\STM32\Program\1.11_Odchudzanie\um0427\FWLib\library\src/stm32f10x_i2c.c:618
   8:	f001 01fe 	and.w	r1, r1, #254	; 0xfe
D:\STM32\Program\1.11_Odchudzanie\um0427\FWLib\library\src/stm32f10x_i2c.c:621
   c:	8201      	strh	r1, [r0, #16]
D:\STM32\Program\1.11_Odchudzanie\um0427\FWLib\library\src/stm32f10x_i2c.c:622
   e:	4770      	bx	lr
Disassembly of section .text.I2C_ReadRegister:

00000000 <I2C_ReadRegister>:
I2C_ReadRegister():
D:\STM32\Program\1.11_Odchudzanie\um0427\FWLib\library\src/stm32f10x_i2c.c:642
   0:	b082      	sub	sp, #8
D:\STM32\Program\1.11_Odchudzanie\um0427\FWLib\library\src/stm32f10x_i2c.c:648
   2:	9b01      	ldr	r3, [sp, #4]
   4:	5ac8      	ldrh	r0, [r1, r3]
D:\STM32\Program\1.11_Odchudzanie\um0427\FWLib\library\src/stm32f10x_i2c.c:649
   6:	b280      	uxth	r0, r0
   8:	b002      	add	sp, #8
   a:	4770      	bx	lr
Disassembly of section .text.I2C_SoftwareResetCmd:

00000000 <I2C_SoftwareResetCmd>:
I2C_SoftwareResetCmd():
D:\STM32\Program\1.11_Odchudzanie\um0427\FWLib\library\src/stm32f10x_i2c.c:666
   0:	b131      	cbz	r1, 10 <I2C_SoftwareResetCmd+0x10>
D:\STM32\Program\1.11_Odchudzanie\um0427\FWLib\library\src/stm32f10x_i2c.c:669
   2:	8803      	ldrh	r3, [r0, #0]
   4:	ea6f 4343 	mvn.w	r3, r3, lsl #17
   8:	ea6f 4353 	mvn.w	r3, r3, lsr #17
   c:	b29b      	uxth	r3, r3
   e:	e002      	b.n	16 <I2C_SoftwareResetCmd+0x16>
D:\STM32\Program\1.11_Odchudzanie\um0427\FWLib\library\src/stm32f10x_i2c.c:674
  10:	8803      	ldrh	r3, [r0, #0]
  12:	045b      	lsls	r3, r3, #17
  14:	0c5b      	lsrs	r3, r3, #17
  16:	8003      	strh	r3, [r0, #0]
D:\STM32\Program\1.11_Odchudzanie\um0427\FWLib\library\src/stm32f10x_i2c.c:676
  18:	4770      	bx	lr
  1a:	46c0      	nop			(mov r8, r8)
Disassembly of section .text.I2C_SMBusAlertConfig:

00000000 <I2C_SMBusAlertConfig>:
I2C_SMBusAlertConfig():
D:\STM32\Program\1.11_Odchudzanie\um0427\FWLib\library\src/stm32f10x_i2c.c:695
   0:	f5b1 5f00 	cmp.w	r1, #8192	; 0x2000
   4:	d104      	bne.n	10 <I2C_SMBusAlertConfig+0x10>
D:\STM32\Program\1.11_Odchudzanie\um0427\FWLib\library\src/stm32f10x_i2c.c:698
   6:	8803      	ldrh	r3, [r0, #0]
   8:	b29b      	uxth	r3, r3
   a:	f443 5300 	orr.w	r3, r3, #8192	; 0x2000
   e:	e004      	b.n	1a <I2C_SMBusAlertConfig+0x1a>
D:\STM32\Program\1.11_Odchudzanie\um0427\FWLib\library\src/stm32f10x_i2c.c:703
  10:	8803      	ldrh	r3, [r0, #0]
  12:	f423 5300 	bic.w	r3, r3, #8192	; 0x2000
  16:	041b      	lsls	r3, r3, #16
  18:	0c1b      	lsrs	r3, r3, #16
  1a:	8003      	strh	r3, [r0, #0]
D:\STM32\Program\1.11_Odchudzanie\um0427\FWLib\library\src/stm32f10x_i2c.c:705
  1c:	4770      	bx	lr
  1e:	46c0      	nop			(mov r8, r8)
Disassembly of section .text.I2C_TransmitPEC:

00000000 <I2C_TransmitPEC>:
I2C_TransmitPEC():
D:\STM32\Program\1.11_Odchudzanie\um0427\FWLib\library\src/stm32f10x_i2c.c:722
   0:	b121      	cbz	r1, c <I2C_TransmitPEC+0xc>
D:\STM32\Program\1.11_Odchudzanie\um0427\FWLib\library\src/stm32f10x_i2c.c:725
   2:	8803      	ldrh	r3, [r0, #0]
   4:	b29b      	uxth	r3, r3
   6:	f443 5380 	orr.w	r3, r3, #4096	; 0x1000
   a:	e004      	b.n	16 <I2C_TransmitPEC+0x16>
D:\STM32\Program\1.11_Odchudzanie\um0427\FWLib\library\src/stm32f10x_i2c.c:730
   c:	8803      	ldrh	r3, [r0, #0]
   e:	f423 5380 	bic.w	r3, r3, #4096	; 0x1000
  12:	041b      	lsls	r3, r3, #16
  14:	0c1b      	lsrs	r3, r3, #16
  16:	8003      	strh	r3, [r0, #0]
D:\STM32\Program\1.11_Odchudzanie\um0427\FWLib\library\src/stm32f10x_i2c.c:732
  18:	4770      	bx	lr
  1a:	46c0      	nop			(mov r8, r8)
Disassembly of section .text.I2C_PECPositionConfig:

00000000 <I2C_PECPositionConfig>:
I2C_PECPositionConfig():
D:\STM32\Program\1.11_Odchudzanie\um0427\FWLib\library\src/stm32f10x_i2c.c:753
   0:	f5b1 6f00 	cmp.w	r1, #2048	; 0x800
   4:	d104      	bne.n	10 <I2C_PECPositionConfig+0x10>
D:\STM32\Program\1.11_Odchudzanie\um0427\FWLib\library\src/stm32f10x_i2c.c:756
   6:	8803      	ldrh	r3, [r0, #0]
   8:	b29b      	uxth	r3, r3
   a:	f443 6300 	orr.w	r3, r3, #2048	; 0x800
   e:	e004      	b.n	1a <I2C_PECPositionConfig+0x1a>
D:\STM32\Program\1.11_Odchudzanie\um0427\FWLib\library\src/stm32f10x_i2c.c:761
  10:	8803      	ldrh	r3, [r0, #0]
  12:	f423 6300 	bic.w	r3, r3, #2048	; 0x800
  16:	041b      	lsls	r3, r3, #16
  18:	0c1b      	lsrs	r3, r3, #16
  1a:	8003      	strh	r3, [r0, #0]
D:\STM32\Program\1.11_Odchudzanie\um0427\FWLib\library\src/stm32f10x_i2c.c:763
  1c:	4770      	bx	lr
  1e:	46c0      	nop			(mov r8, r8)
Disassembly of section .text.I2C_CalculatePEC:

00000000 <I2C_CalculatePEC>:
I2C_CalculatePEC():
D:\STM32\Program\1.11_Odchudzanie\um0427\FWLib\library\src/stm32f10x_i2c.c:781
   0:	b121      	cbz	r1, c <I2C_CalculatePEC+0xc>
D:\STM32\Program\1.11_Odchudzanie\um0427\FWLib\library\src/stm32f10x_i2c.c:784
   2:	8803      	ldrh	r3, [r0, #0]
   4:	b29b      	uxth	r3, r3
   6:	f043 0320 	orr.w	r3, r3, #32	; 0x20
   a:	e004      	b.n	16 <I2C_CalculatePEC+0x16>
D:\STM32\Program\1.11_Odchudzanie\um0427\FWLib\library\src/stm32f10x_i2c.c:789
   c:	8803      	ldrh	r3, [r0, #0]
   e:	f023 0320 	bic.w	r3, r3, #32	; 0x20
  12:	041b      	lsls	r3, r3, #16
  14:	0c1b      	lsrs	r3, r3, #16
  16:	8003      	strh	r3, [r0, #0]
D:\STM32\Program\1.11_Odchudzanie\um0427\FWLib\library\src/stm32f10x_i2c.c:791
  18:	4770      	bx	lr
  1a:	46c0      	nop			(mov r8, r8)
Disassembly of section .text.I2C_GetPEC:

00000000 <I2C_GetPEC>:
I2C_GetPEC():
D:\STM32\Program\1.11_Odchudzanie\um0427\FWLib\library\src/stm32f10x_i2c.c:806
   0:	8b00      	ldrh	r0, [r0, #24]
D:\STM32\Program\1.11_Odchudzanie\um0427\FWLib\library\src/stm32f10x_i2c.c:807
   2:	f3c0 2007 	ubfx	r0, r0, #8, #8
   6:	4770      	bx	lr
Disassembly of section .text.I2C_ARPCmd:

00000000 <I2C_ARPCmd>:
I2C_ARPCmd():
D:\STM32\Program\1.11_Odchudzanie\um0427\FWLib\library\src/stm32f10x_i2c.c:824
   0:	b121      	cbz	r1, c <I2C_ARPCmd+0xc>
D:\STM32\Program\1.11_Odchudzanie\um0427\FWLib\library\src/stm32f10x_i2c.c:827
   2:	8803      	ldrh	r3, [r0, #0]
   4:	b29b      	uxth	r3, r3
   6:	f043 0310 	orr.w	r3, r3, #16	; 0x10
   a:	e004      	b.n	16 <I2C_ARPCmd+0x16>
D:\STM32\Program\1.11_Odchudzanie\um0427\FWLib\library\src/stm32f10x_i2c.c:832
   c:	8803      	ldrh	r3, [r0, #0]
   e:	f023 0310 	bic.w	r3, r3, #16	; 0x10
  12:	041b      	lsls	r3, r3, #16
  14:	0c1b      	lsrs	r3, r3, #16
  16:	8003      	strh	r3, [r0, #0]
D:\STM32\Program\1.11_Odchudzanie\um0427\FWLib\library\src/stm32f10x_i2c.c:834
  18:	4770      	bx	lr
  1a:	46c0      	nop			(mov r8, r8)
Disassembly of section .text.I2C_StretchClockCmd:

00000000 <I2C_StretchClockCmd>:
I2C_StretchClockCmd():
D:\STM32\Program\1.11_Odchudzanie\um0427\FWLib\library\src/stm32f10x_i2c.c:851
   0:	b921      	cbnz	r1, c <I2C_StretchClockCmd+0xc>
D:\STM32\Program\1.11_Odchudzanie\um0427\FWLib\library\src/stm32f10x_i2c.c:854
   2:	8803      	ldrh	r3, [r0, #0]
   4:	b29b      	uxth	r3, r3
   6:	f043 0380 	orr.w	r3, r3, #128	; 0x80
   a:	e004      	b.n	16 <I2C_StretchClockCmd+0x16>
D:\STM32\Program\1.11_Odchudzanie\um0427\FWLib\library\src/stm32f10x_i2c.c:859
   c:	8803      	ldrh	r3, [r0, #0]
   e:	f023 0380 	bic.w	r3, r3, #128	; 0x80
  12:	041b      	lsls	r3, r3, #16
  14:	0c1b      	lsrs	r3, r3, #16
  16:	8003      	strh	r3, [r0, #0]
D:\STM32\Program\1.11_Odchudzanie\um0427\FWLib\library\src/stm32f10x_i2c.c:861
  18:	4770      	bx	lr
  1a:	46c0      	nop			(mov r8, r8)
Disassembly of section .text.I2C_FastModeDutyCycleConfig:

00000000 <I2C_FastModeDutyCycleConfig>:
I2C_FastModeDutyCycleConfig():
D:\STM32\Program\1.11_Odchudzanie\um0427\FWLib\library\src/stm32f10x_i2c.c:880
   0:	f5b1 4f80 	cmp.w	r1, #16384	; 0x4000
   4:	d005      	beq.n	12 <I2C_FastModeDutyCycleConfig+0x12>
D:\STM32\Program\1.11_Odchudzanie\um0427\FWLib\library\src/stm32f10x_i2c.c:883
   6:	8b83      	ldrh	r3, [r0, #28]
   8:	f423 4380 	bic.w	r3, r3, #16384	; 0x4000
   c:	041b      	lsls	r3, r3, #16
   e:	0c1b      	lsrs	r3, r3, #16
  10:	e003      	b.n	1a <I2C_FastModeDutyCycleConfig+0x1a>
D:\STM32\Program\1.11_Odchudzanie\um0427\FWLib\library\src/stm32f10x_i2c.c:888
  12:	8b83      	ldrh	r3, [r0, #28]
  14:	b29b      	uxth	r3, r3
  16:	f443 4380 	orr.w	r3, r3, #16384	; 0x4000
  1a:	8383      	strh	r3, [r0, #28]
D:\STM32\Program\1.11_Odchudzanie\um0427\FWLib\library\src/stm32f10x_i2c.c:890
  1c:	4770      	bx	lr
  1e:	46c0      	nop			(mov r8, r8)
Disassembly of section .text.I2C_GetLastEvent:

00000000 <I2C_GetLastEvent>:
I2C_GetLastEvent():
D:\STM32\Program\1.11_Odchudzanie\um0427\FWLib\library\src/stm32f10x_i2c.c:900
   0:	4603      	mov	r3, r0
D:\STM32\Program\1.11_Odchudzanie\um0427\FWLib\library\src/stm32f10x_i2c.c:908
   2:	8a80      	ldrh	r0, [r0, #20]
D:\STM32\Program\1.11_Odchudzanie\um0427\FWLib\library\src/stm32f10x_i2c.c:909
   4:	8b1b      	ldrh	r3, [r3, #24]
D:\STM32\Program\1.11_Odchudzanie\um0427\FWLib\library\src/stm32f10x_i2c.c:908
   6:	b280      	uxth	r0, r0
D:\STM32\Program\1.11_Odchudzanie\um0427\FWLib\library\src/stm32f10x_i2c.c:909
   8:	ea40 4003 	orr.w	r0, r0, r3, lsl #16
D:\STM32\Program\1.11_Odchudzanie\um0427\FWLib\library\src/stm32f10x_i2c.c:917
   c:	f020 407f 	bic.w	r0, r0, #4278190080	; 0xff000000
  10:	4770      	bx	lr
  12:	46c0      	nop			(mov r8, r8)
Disassembly of section .text.I2C_CheckEvent:

00000000 <I2C_CheckEvent>:
I2C_CheckEvent():
D:\STM32\Program\1.11_Odchudzanie\um0427\FWLib\library\src/stm32f10x_i2c.c:942
   0:	4603      	mov	r3, r0
D:\STM32\Program\1.11_Odchudzanie\um0427\FWLib\library\src/stm32f10x_i2c.c:952
   2:	8a80      	ldrh	r0, [r0, #20]
D:\STM32\Program\1.11_Odchudzanie\um0427\FWLib\library\src/stm32f10x_i2c.c:953
   4:	8b1b      	ldrh	r3, [r3, #24]
D:\STM32\Program\1.11_Odchudzanie\um0427\FWLib\library\src/stm32f10x_i2c.c:952
   6:	b280      	uxth	r0, r0
D:\STM32\Program\1.11_Odchudzanie\um0427\FWLib\library\src/stm32f10x_i2c.c:953
   8:	ea40 4003 	orr.w	r0, r0, r3, lsl #16
   c:	f020 407f 	bic.w	r0, r0, #4278190080	; 0xff000000
D:\STM32\Program\1.11_Odchudzanie\um0427\FWLib\library\src/stm32f10x_i2c.c:973
  10:	4288      	cmp	r0, r1
  12:	bf14      	ite	ne
  14:	2000      	movne	r0, #0
  16:	2001      	moveq	r0, #1
  18:	4770      	bx	lr
  1a:	46c0      	nop			(mov r8, r8)
Disassembly of section .text.I2C_GetFlagStatus:

00000000 <I2C_GetFlagStatus>:
I2C_GetFlagStatus():
D:\STM32\Program\1.11_Odchudzanie\um0427\FWLib\library\src/stm32f10x_i2c.c:1007
   0:	b082      	sub	sp, #8
D:\STM32\Program\1.11_Odchudzanie\um0427\FWLib\library\src/stm32f10x_i2c.c:1022
   2:	f021 427f 	bic.w	r2, r1, #4278190080	; 0xff000000
D:\STM32\Program\1.11_Odchudzanie\um0427\FWLib\library\src/stm32f10x_i2c.c:1024
   6:	0f09      	lsrs	r1, r1, #28
D:\STM32\Program\1.11_Odchudzanie\um0427\FWLib\library\src/stm32f10x_i2c.c:1007
   8:	9001      	str	r0, [sp, #4]
D:\STM32\Program\1.11_Odchudzanie\um0427\FWLib\library\src/stm32f10x_i2c.c:1024
   a:	d001      	beq.n	10 <I2C_GetFlagStatus+0x10>
D:\STM32\Program\1.11_Odchudzanie\um0427\FWLib\library\src/stm32f10x_i2c.c:1027
   c:	3014      	adds	r0, #20
   e:	e001      	b.n	14 <I2C_GetFlagStatus+0x14>
D:\STM32\Program\1.11_Odchudzanie\um0427\FWLib\library\src/stm32f10x_i2c.c:1032
  10:	0c12      	lsrs	r2, r2, #16
D:\STM32\Program\1.11_Odchudzanie\um0427\FWLib\library\src/stm32f10x_i2c.c:1034
  12:	3018      	adds	r0, #24
D:\STM32\Program\1.11_Odchudzanie\um0427\FWLib\library\src/stm32f10x_i2c.c:1037
  14:	6803      	ldr	r3, [r0, #0]
  16:	4213      	tst	r3, r2
D:\STM32\Program\1.11_Odchudzanie\um0427\FWLib\library\src/stm32f10x_i2c.c:1050
  18:	bf0c      	ite	eq
  1a:	2000      	moveq	r0, #0
  1c:	2001      	movne	r0, #1
  1e:	b002      	add	sp, #8
  20:	4770      	bx	lr
  22:	46c0      	nop			(mov r8, r8)
Disassembly of section .text.I2C_ClearFlag:

00000000 <I2C_ClearFlag>:
I2C_ClearFlag():
D:\STM32\Program\1.11_Odchudzanie\um0427\FWLib\library\src/stm32f10x_i2c.c:1104
   0:	43c9      	mvns	r1, r1
   2:	b289      	uxth	r1, r1
   4:	8281      	strh	r1, [r0, #20]
D:\STM32\Program\1.11_Odchudzanie\um0427\FWLib\library\src/stm32f10x_i2c.c:1105
   6:	4770      	bx	lr
Disassembly of section .text.I2C_GetITStatus:

00000000 <I2C_GetITStatus>:
I2C_GetITStatus():
D:\STM32\Program\1.11_Odchudzanie\um0427\FWLib\library\src/stm32f10x_i2c.c:1132
   0:	8883      	ldrh	r3, [r0, #4]
   2:	b29a      	uxth	r2, r3
D:\STM32\Program\1.11_Odchudzanie\um0427\FWLib\library\src/stm32f10x_i2c.c:1147
   4:	8a83      	ldrh	r3, [r0, #20]
   6:	b29b      	uxth	r3, r3
   8:	ea13 0001 	ands.w	r0, r3, r1
   c:	d006      	beq.n	1c <I2C_GetITStatus+0x1c>
   e:	f001 63e0 	and.w	r3, r1, #117440512	; 0x7000000
  12:	ea12 4313 	ands.w	r3, r2, r3, lsr #16
  16:	bf0c      	ite	eq
  18:	2000      	moveq	r0, #0
  1a:	2001      	movne	r0, #1
D:\STM32\Program\1.11_Odchudzanie\um0427\FWLib\library\src/stm32f10x_i2c.c:1159
  1c:	4770      	bx	lr
  1e:	46c0      	nop			(mov r8, r8)
Disassembly of section .text.I2C_ClearITPendingBit:

00000000 <I2C_ClearITPendingBit>:
I2C_ClearITPendingBit():
D:\STM32\Program\1.11_Odchudzanie\um0427\FWLib\library\src/stm32f10x_i2c.c:1202
   0:	43c9      	mvns	r1, r1
   2:	b289      	uxth	r1, r1
   4:	8281      	strh	r1, [r0, #20]
D:\STM32\Program\1.11_Odchudzanie\um0427\FWLib\library\src/stm32f10x_i2c.c:1214
   6:	4770      	bx	lr
Disassembly of section .text.I2C_Init:

00000000 <I2C_Init>:
I2C_Init():
D:\STM32\Program\1.11_Odchudzanie\um0427\FWLib\library\src/stm32f10x_i2c.c:150
   0:	b570      	push	{r4, r5, r6, lr}
   2:	b086      	sub	sp, #24
   4:	4605      	mov	r5, r0
D:\STM32\Program\1.11_Odchudzanie\um0427\FWLib\library\src/stm32f10x_i2c.c:167
   6:	8884      	ldrh	r4, [r0, #4]
D:\STM32\Program\1.11_Odchudzanie\um0427\FWLib\library\src/stm32f10x_i2c.c:171
   8:	a801      	add	r0, sp, #4
D:\STM32\Program\1.11_Odchudzanie\um0427\FWLib\library\src/stm32f10x_i2c.c:150
   a:	460e      	mov	r6, r1
D:\STM32\Program\1.11_Odchudzanie\um0427\FWLib\library\src/stm32f10x_i2c.c:171
   c:	f7ff fffe 	bl	0 <RCC_GetClocksFreq>
D:\STM32\Program\1.11_Odchudzanie\um0427\FWLib\library\src/stm32f10x_i2c.c:172
  10:	9803      	ldr	r0, [sp, #12]
D:\STM32\Program\1.11_Odchudzanie\um0427\FWLib\library\src/stm32f10x_i2c.c:174
  12:	4b31      	ldr	r3, [pc, #196]	(d8 <RCC_GetClocksFreq+0xd8>)
D:\STM32\Program\1.11_Odchudzanie\um0427\FWLib\library\src/stm32f10x_i2c.c:169
  14:	f024 043f 	bic.w	r4, r4, #63	; 0x3f
  18:	0424      	lsls	r4, r4, #16
D:\STM32\Program\1.11_Odchudzanie\um0427\FWLib\library\src/stm32f10x_i2c.c:174
  1a:	fbb0 f3f3 	udiv	r3, r0, r3
D:\STM32\Program\1.11_Odchudzanie\um0427\FWLib\library\src/stm32f10x_i2c.c:169
  1e:	0c24      	lsrs	r4, r4, #16
D:\STM32\Program\1.11_Odchudzanie\um0427\FWLib\library\src/stm32f10x_i2c.c:174
  20:	fa1f fe83 	uxth.w	lr, r3
D:\STM32\Program\1.11_Odchudzanie\um0427\FWLib\library\src/stm32f10x_i2c.c:175
  24:	ea4e 0404 	orr.w	r4, lr, r4
D:\STM32\Program\1.11_Odchudzanie\um0427\FWLib\library\src/stm32f10x_i2c.c:177
  28:	80ac      	strh	r4, [r5, #4]
D:\STM32\Program\1.11_Odchudzanie\um0427\FWLib\library\src/stm32f10x_i2c.c:181
  2a:	882b      	ldrh	r3, [r5, #0]
D:\STM32\Program\1.11_Odchudzanie\um0427\FWLib\library\src/stm32f10x_i2c.c:188
  2c:	68f1      	ldr	r1, [r6, #12]
D:\STM32\Program\1.11_Odchudzanie\um0427\FWLib\library\src/stm32f10x_i2c.c:181
  2e:	f023 0301 	bic.w	r3, r3, #1	; 0x1
  32:	041b      	lsls	r3, r3, #16
  34:	0c1b      	lsrs	r3, r3, #16
  36:	802b      	strh	r3, [r5, #0]
D:\STM32\Program\1.11_Odchudzanie\um0427\FWLib\library\src/stm32f10x_i2c.c:188
  38:	4b28      	ldr	r3, [pc, #160]	(dc <RCC_GetClocksFreq+0xdc>)
  3a:	4299      	cmp	r1, r3
  3c:	d80c      	bhi.n	58 <RCC_GetClocksFreq+0x58>
D:\STM32\Program\1.11_Odchudzanie\um0427\FWLib\library\src/stm32f10x_i2c.c:191
  3e:	004a      	lsls	r2, r1, #1
  40:	fbb0 f2f2 	udiv	r2, r0, r2
D:\STM32\Program\1.11_Odchudzanie\um0427\FWLib\library\src/stm32f10x_i2c.c:201
  44:	f10e 0301 	add.w	r3, lr, #1	; 0x1
D:\STM32\Program\1.11_Odchudzanie\um0427\FWLib\library\src/stm32f10x_i2c.c:191
  48:	b292      	uxth	r2, r2
D:\STM32\Program\1.11_Odchudzanie\um0427\FWLib\library\src/stm32f10x_i2c.c:201
  4a:	b29b      	uxth	r3, r3
  4c:	842b      	strh	r3, [r5, #32]
  4e:	2a03      	cmp	r2, #3
  50:	bf8c      	ite	hi
  52:	4611      	movhi	r1, r2
  54:	2104      	movls	r1, #4
  56:	e025      	b.n	a4 <RCC_GetClocksFreq+0xa4>
D:\STM32\Program\1.11_Odchudzanie\um0427\FWLib\library\src/stm32f10x_i2c.c:206
  58:	8872      	ldrh	r2, [r6, #2]
  5a:	f64b 73ff 	movw	r3, #49151	; 0xbfff
  5e:	429a      	cmp	r2, r3
  60:	d106      	bne.n	70 <RCC_GetClocksFreq+0x70>
D:\STM32\Program\1.11_Odchudzanie\um0427\FWLib\library\src/stm32f10x_i2c.c:209
  62:	2303      	movs	r3, #3
  64:	fb01 f303 	mul.w	r3, r1, r3
  68:	fbb0 f3f3 	udiv	r3, r0, r3
  6c:	b29a      	uxth	r2, r3
  6e:	e007      	b.n	80 <RCC_GetClocksFreq+0x80>
D:\STM32\Program\1.11_Odchudzanie\um0427\FWLib\library\src/stm32f10x_i2c.c:214
  70:	2319      	movs	r3, #25
  72:	fb01 f303 	mul.w	r3, r1, r3
  76:	fbb0 f3f3 	udiv	r3, r0, r3
  7a:	b29b      	uxth	r3, r3
D:\STM32\Program\1.11_Odchudzanie\um0427\FWLib\library\src/stm32f10x_i2c.c:216
  7c:	f443 4280 	orr.w	r2, r3, #16384	; 0x4000
D:\STM32\Program\1.11_Odchudzanie\um0427\FWLib\library\src/stm32f10x_i2c.c:219
  80:	0513      	lsls	r3, r2, #20
  82:	0d1b      	lsrs	r3, r3, #20
  84:	b90b      	cbnz	r3, 8a <RCC_GetClocksFreq+0x8a>
D:\STM32\Program\1.11_Odchudzanie\um0427\FWLib\library\src/stm32f10x_i2c.c:222
  86:	f042 0201 	orr.w	r2, r2, #1	; 0x1
D:\STM32\Program\1.11_Odchudzanie\um0427\FWLib\library\src/stm32f10x_i2c.c:227
  8a:	f44f 7396 	mov.w	r3, #300	; 0x12c
  8e:	fb0e f303 	mul.w	r3, lr, r3
D:\STM32\Program\1.11_Odchudzanie\um0427\FWLib\library\src/stm32f10x_i2c.c:225
  92:	f442 4100 	orr.w	r1, r2, #32768	; 0x8000
D:\STM32\Program\1.11_Odchudzanie\um0427\FWLib\library\src/stm32f10x_i2c.c:227
  96:	f44f 727a 	mov.w	r2, #1000	; 0x3e8
  9a:	fb93 f3f2 	sdiv	r3, r3, r2
  9e:	3301      	adds	r3, #1
  a0:	b29b      	uxth	r3, r3
  a2:	842b      	strh	r3, [r5, #32]
D:\STM32\Program\1.11_Odchudzanie\um0427\FWLib\library\src/stm32f10x_i2c.c:230
  a4:	83a9      	strh	r1, [r5, #28]
D:\STM32\Program\1.11_Odchudzanie\um0427\FWLib\library\src/stm32f10x_i2c.c:233
  a6:	882b      	ldrh	r3, [r5, #0]
  a8:	b29b      	uxth	r3, r3
  aa:	f043 0301 	orr.w	r3, r3, #1	; 0x1
  ae:	802b      	strh	r3, [r5, #0]
D:\STM32\Program\1.11_Odchudzanie\um0427\FWLib\library\src/stm32f10x_i2c.c:237
  b0:	882b      	ldrh	r3, [r5, #0]
D:\STM32\Program\1.11_Odchudzanie\um0427\FWLib\library\src/stm32f10x_i2c.c:243
  b2:	88f2      	ldrh	r2, [r6, #6]
D:\STM32\Program\1.11_Odchudzanie\um0427\FWLib\library\src/stm32f10x_i2c.c:239
  b4:	f423 6380 	bic.w	r3, r3, #1024	; 0x400
D:\STM32\Program\1.11_Odchudzanie\um0427\FWLib\library\src/stm32f10x_i2c.c:243
  b8:	8831      	ldrh	r1, [r6, #0]
D:\STM32\Program\1.11_Odchudzanie\um0427\FWLib\library\src/stm32f10x_i2c.c:239
  ba:	f023 030a 	bic.w	r3, r3, #10	; 0xa
  be:	041b      	lsls	r3, r3, #16
D:\STM32\Program\1.11_Odchudzanie\um0427\FWLib\library\src/stm32f10x_i2c.c:243
  c0:	430a      	orrs	r2, r1
D:\STM32\Program\1.11_Odchudzanie\um0427\FWLib\library\src/stm32f10x_i2c.c:239
  c2:	0c1b      	lsrs	r3, r3, #16
D:\STM32\Program\1.11_Odchudzanie\um0427\FWLib\library\src/stm32f10x_i2c.c:243
  c4:	4313      	orrs	r3, r2
  c6:	b29b      	uxth	r3, r3
D:\STM32\Program\1.11_Odchudzanie\um0427\FWLib\library\src/stm32f10x_i2c.c:245
  c8:	802b      	strh	r3, [r5, #0]
D:\STM32\Program\1.11_Odchudzanie\um0427\FWLib\library\src/stm32f10x_i2c.c:249
  ca:	88b3      	ldrh	r3, [r6, #4]
  cc:	8932      	ldrh	r2, [r6, #8]
  ce:	4313      	orrs	r3, r2
  d0:	b29b      	uxth	r3, r3
  d2:	812b      	strh	r3, [r5, #8]
D:\STM32\Program\1.11_Odchudzanie\um0427\FWLib\library\src/stm32f10x_i2c.c:250
  d4:	b006      	add	sp, #24
  d6:	bd70      	pop	{r4, r5, r6, pc}
  d8:	000f4240 	.word	0x000f4240
  dc:	000186a0 	.word	0x000186a0
Disassembly of section .text.I2C_DeInit:

00000000 <I2C_DeInit>:
I2C_DeInit():
D:\STM32\Program\1.11_Odchudzanie\um0427\FWLib\library\src/stm32f10x_i2c.c:113
   0:	b507      	push	{r0, r1, r2, lr}
D:\STM32\Program\1.11_Odchudzanie\um0427\FWLib\library\src/stm32f10x_i2c.c:117
   2:	4b0e      	ldr	r3, [pc, #56]	(3c <I2C_DeInit+0x3c>)
D:\STM32\Program\1.11_Odchudzanie\um0427\FWLib\library\src/stm32f10x_i2c.c:113
   4:	9001      	str	r0, [sp, #4]
D:\STM32\Program\1.11_Odchudzanie\um0427\FWLib\library\src/stm32f10x_i2c.c:117
   6:	4298      	cmp	r0, r3
   8:	d004      	beq.n	14 <I2C_DeInit+0x14>
   a:	f503 6380 	add.w	r3, r3, #1024	; 0x400
   e:	4298      	cmp	r0, r3
  10:	d008      	beq.n	24 <I2C_DeInit+0x24>
  12:	e011      	b.n	38 <I2C_DeInit+0x38>
D:\STM32\Program\1.11_Odchudzanie\um0427\FWLib\library\src/stm32f10x_i2c.c:121
  14:	f44f 1000 	mov.w	r0, #2097152	; 0x200000
  18:	2101      	movs	r1, #1
  1a:	f7ff fffe 	bl	0 <RCC_APB1PeriphResetCmd>
D:\STM32\Program\1.11_Odchudzanie\um0427\FWLib\library\src/stm32f10x_i2c.c:123
  1e:	f44f 1000 	mov.w	r0, #2097152	; 0x200000
  22:	e006      	b.n	32 <I2C_DeInit+0x32>
D:\STM32\Program\1.11_Odchudzanie\um0427\FWLib\library\src/stm32f10x_i2c.c:128
  24:	f44f 0080 	mov.w	r0, #4194304	; 0x400000
  28:	2101      	movs	r1, #1
  2a:	f7ff fffe 	bl	0 <RCC_APB1PeriphResetCmd>
D:\STM32\Program\1.11_Odchudzanie\um0427\FWLib\library\src/stm32f10x_i2c.c:130
  2e:	f44f 0080 	mov.w	r0, #4194304	; 0x400000
  32:	2100      	movs	r1, #0
  34:	f7ff fffe 	bl	0 <RCC_APB1PeriphResetCmd>
D:\STM32\Program\1.11_Odchudzanie\um0427\FWLib\library\src/stm32f10x_i2c.c:136
  38:	bd0e      	pop	{r1, r2, r3, pc}
  3a:	46c0      	nop			(mov r8, r8)
  3c:	40005400 	.word	0x40005400
